S02F0000643A5C2D70726F6A6563742D5C726372786465636F6465725C61736D5C726372786465636F6465722E6D6F7488
S1130000F8C011C01895189584C01895B8C01895F3
S11300101895189518951895189518951895189574
S11300201895189518959F938F930F930FB70F9367
S113003070FD14C093E080E28A179B0758F59AE09C
S113004080EF8A179B0730F171603327BB27AA27FB
S11300500F910FBF0F918F919F91189590E08EEBA8
S11300608A179B07B8F491E088EB8A179B0790F0F6
S11300706030D9F06A95339533953E3019F47E7F1C
S1130080EE24DD24BB27AA270F910FBF0F918F9178
S11300909F9118957E7F726067E0BB27AA270F9116
S11300A00FBF0F918F919F9118951127552705E048
S11300B003BFE0E673FDEC0DE30F91918081A80F7F
S11300C0B91F8894B795A795E0E673FDEC0DE30F8F
S11300D0B193A083DA0EEB1E339533953E3089F449
S11300E07E7F9FE08CE38D199E09E0E673FDEC0DA5
S11300F0E30F9193808308E070277D7F7B7FEE245C
S1130100DD24BB27AA270F910FBF0F918F919F91D9
S113011018959F938F930F930FB70F931196219672
S1130120403011F401E008BB08E07027E0E673FDFD
S1130130EC0DE40F9191808108E070278C179D07E6
S113014030F00F910FBF0F918F919F9118954E3002
S113015069F008B3000F08BB43954395DD27CC270E
S11301600F910FBF0F918F919F9118954427DD2711
S1130170CC270F910FBF0F918F919F9118959F934B
S11301808F930F930FB70F93103539F013950F9189
S11301900FBF0F918F919F9118957460E199FECFD5
S11301A000E0050F0EBBE09A9DB3E199FECF00E09D
S11301B0050F03950EBBE09A8DB3E0E673FDEC0DDD
S11301C0E50F9193808308E07027E0E673FDEC0D62
S11301D0E50F9193808308E0702753955395503130
S11301E011F4002703BF0F910FBF0F918F919F91BF
S11301F018950FED0DBFF8940FEF07BB8C9A8D9AED
S1130200929A939A00E40BBF02E005BF02E409BF8F
S113021044273327552711277727FF27BB27AA27EA
S1130220DD27CC2704E1C02EE199FECF00E0020FC8
S11302300EBBE09A9DB3E199FECF00E0020F039557
S11302400EBBE09A8DB3E0E673FDEC0DE20F9193E3
S1130250808308E07027E0E673FDEC0DE20F9193D4
S1130260808308E07027239523952031E9F67E7F6B
S1130270726067E0789400E00BBD04E60ABD09E013
S11302800EBD05E003BF72FD02C0959801C0959AAA
S113029071FD02C0949802C0949AF5CF8399FF240B
S11302A0F39489F7F894959A002708BB222708E06D
S11302B07027E0E673FDEC0DE20F91918081E199E6
S11302C0FECF00E0020F0EBB9DBBE29AE19AE199DA
S11302D0FECF00E0020F03950EBB8DBBE29AE19ABC
S11302E023952395203129F7959808E07027839B5F
S10902F0FECF7894C8CF94
S5030030CC
S9030000FC
